:100000006F00804B000000000A0300000E03000098
:1000100000000000000000000000000000000000E0
:1000200000000000000000000000000000000000D0
:10003000C40300000000000088040000000000006D
:100040008A0400008C0400008E040000900400006C
:10005000920400009404000096040000980400003C
:100060009A0400009C0400009E040000A00400000C
:10007000A2040000A4040000A6040000A8040000DC
:10008000AA040000AC040000AE040000B0040000AC
:10009000B2040000B4040000B60400000100000037
:1000A000B7070020938787009823A1466308D706E7
:1000B000EF02C03B71112AC0131527003A9523A205
:1000C00027000E05B6973E95138105149D260DE574
:1000D0003707002013078700142303214700939755
:1000E00026000246B6978E07BA97850690D723A6B4
:1000F000070214A3110149A6370400201304840049
:100100000347841493172700BA978E07A297C857FE
:100110009857029789451305041525268280B7074D
:1001200000209387870003C707171DC3EF02003421
:1001300003C787141385870093172700BA978E0784
:100140003E95C52C09E5854513850195DD2C2DA629
:100150008280EF02A031370400201304840083243E
:100160004417711183274417858F63E4A700110199
:1001700021A62AC06D370245F5B7EF02202F3717A9
:1001800002401C4F7111054593E707011CCFB717BB
:10019000014090433D4381478D42A1453317F5000F
:1001A0001377F7FD01EF939627003317D30013471A
:1001B000F7FF718FB396D20033E6E6008507E39F21
:1001C000B7FC3717014010C33EC0371401409304F9
:1001D00000021305401F04C8AD3F1305401F44C86B
:1001E0008D3F8247FD1793F7F70FF9FF110169A4BF
:1001F000EF02C027371702401C4F05453D4393E7E8
:1002000007011CCFB717014090438D428147A1459C
:100210003317F5001377F7FB01EF93962700331799
:10022000D3001347F7FF718FB396D20033E6E60091
:100230008507E39FB7FCB717014090C3371401400F
:100240009304000404C81305803E21371305803E43
:1002500044C80137E5B737050020130585001C2188
:10026000C5C7EF02A020130505157111D922370764
:10027000002013078700854583478714630FB50067
:100280008946630ED50219ED139527003E95230884
:10029000B7160E0521073A956D2285072308071624
:1002A0002304F714B70700209387870083C68714B9
:1002B000982363E4E60023840714110175AA04233C
:1002C0001387F4FF63C8E700FD14B70700202384F9
:1002D0009700C9BF13841700139527003E95931705
:1002E0002400B7050020A2978E07938585000E0590
:1002F0002E95BE9513068002A10521053AC0A12ABC
:1003000002479377F40F7DBF82807300203001A0F5
:10031000B71702409843B706FFFC1367170098C34E
:10032000D843758FD8C39843B706F7FEFD16758F6F
:1003300098C39843B706FCFFFD16758F98C3D84342
:10034000C176FD16758FD8C337079F0098C7984FA1
:100350001367070298CF3717014013070740104370
:100360001376F6F010C310431366060810C309464F
:1003700010CB372702401043719A10C31043136605
:10038000160010C3D843D8C3D843758FD8C3D843F9
:10039000B7060001D8C39843558F98C39843931666
:1003A0006700E3DD06FED843B7160240719BD8C351
:1003B000D84313672700D8C32147DC42B18BE39EA3
:1003C000E7FE8280B70700209387870003A74717BF
:1003D000050723AAE716B7F700E023A2070073007A
:1003E00020303747014081471307078063C4C700A7
:1003F00032858280162393F60604EDDEB386F5007F
:100400009422850756A3DDB737070020130707009E
:10041000AA870843938681EFAA9763EAF600B70696
:1004200000209386464063E4D7001CC382807D553C
:1004300082802320150040C104C5232625000145E4
:10044000828083200500404104450321C50013B587
:1004500015002E9582802A8309CA83830500230014
:1004600073007D16050385056DFA8280511126C043
:1004700022C206C48282010082441244A240310199
:10048000828001A001A001A001A001A001A001A003
:1004900001A001A001A001A001A001A001A001A054
:1004A00001A001A001A001A001A001A001A001A044
:1004B00001A001A001A001A09701002093810135B6
:1004C000170100201301013413050059970500207E
:1004D000938545B317060020130646B363FAC5009B
:1004E0008322050023A0550011059105E3EAC5FE0E
:1004F00017050020130585B1970500209385C5F0E9
:100500006377B500232005001105E36DB5FE930266
:100510000008739002308D42739042809702000071
:10052000938242AE93E2320073905230EFF05FDE7E
:1005300097020000938202017390123473002030FE
:10054000EFF2DFF237040020130484008547232CE8
:10055000F4160567B7E700E023A0E710B7F700E05F
:10056000D8439305C417799BD8C331671307F7B7EE
:1005700098CB23A407003D471305A01798C30D3659
:100580009305C42B1305001F213EF131FDBF000070
:0805900004040020000000003B
:00000001FF
